:020000021000EC
:10F800000C9446FC0C9465FC0C9465FC0C9465FC13
:10F810000C9465FC0C9465FC0C9465FC0C9465FCE4
:10F820000C9465FC0C9465FC0C9465FC0C9465FCD4
:10F830000C9465FC0C9465FC0C9465FC0C9465FCC4
:10F840000C9465FC0C9465FC0C9465FC0C9465FCB4
:10F850000C9465FC0C9465FC0C9465FC0C9465FCA4
:10F860000C9465FC0C9465FC0C9465FC0C9465FC94
:10F870000C9465FC0C9465FC0C9465FC0C9465FC84
:10F880000C9465FC0C9465FC0C9465FC11241FBE63
:10F89000CFEFD0E1DEBFCDBF11E0A0E0B1E0EEE8F8
:10F8A000FFEF01E00BBF02C007900D92A030B1073F
:10F8B000D9F712E0A0E0B1E001C01D92A434B10775
:10F8C000E1F70E947DFF0C94C5FF0C9400FC0F92A1
:10F8D000AF93BF93CF93DF93EF93FF93FC01EA01C4
:10F8E000DB01D895099231961197D9F7FF91EF91E5
:10F8F000DF91CF91BF91AF910F9008950F921F921A
:10F900000F931F93AF93BF93CF93DF93EF93FF9327
:10F91000FC01EA01DB0110E00990199001E04CD0F4
:10F920003296129711F01250B9F7FC0103E044D05F
:10F9300005E042D000E011E0800F911F109759F7C9
:10F94000FF91EF91DF91CF91BF91AF911F910F91F7
:10F950001F900F9008950F931F93EF93FF93FC0157
:10F9600003E02AD000E011E0E00FF11FE617F707EF
:10F97000B9F7FF91EF911F910F9108950F930F9297
:10F9800022D0082E09E018D00F900F9108950F9300
:10F990000F92EF93FF9317D0FC0160936800C89516
:10F9A000802DFF91EF910F900F9108950F930BD041
:10F9B00001E102D00F910895E199FECF0093680014
:10F9C000E895FFFF00000091680000FDFCCF08955E
:10F9D00089E080939900EAE9F0E080818861808382
:10F9E0000895EAE9F0E08081877E8083089580931E
:10F9F0009C0080919B0086FFFCCF80919B008064DF
:10FA000080939B00089580919C00089580919B00B5
:10FA100080780895AC0120E030E00CC080919B001C
:10FA200087FFFCCF80919C00FA01E20FF31F8083D7
:10FA30002F5F3F4F2617370788F381E00895FC01B9
:10FA400020E030E00FC0808180939C0080919B007B
:10FA500086FFFCCF319680919B00806480939B0051
:10FA60002F5F3F4F2617370770F381E008958138E5
:10FA700079F0823818F4803839F408C0823851F0AF
:10FA8000883911F483E0089580E0089582E00895B4
:10FA900081E0089582E108956091400170914101F3
:10FAA000409142025091430220E030E010C0C90171
:10FAB000840F951F9FBB8EBBF901EE5BFE4F8081CB
:10FAC0008DBBE29AE19AE199FECF2F5F3F4F261757
:10FAD000370768F3460F571F509343024093420283
:10FAE000089560914001709141014091420250910E
:10FAF000430220E030E00DC0C901840F951F9FBB79
:10FB00008EBBE09A8DB3F901EE5BFE4F80832F5FD1
:10FB10003F4F2617370780F3460F571F5093430276
:10FB200040934202089540E050E00BC020E030E0F6
:10FB300000002F5F3F4F68E02A3C3607C9F74F5F50
:10FB40005F4F4817590790F3089520914202309172
:10FB5000430237FF03C081E08BBF01C01BBE609131
:10FB600040017091410142E451E0C901880F991FA1
:10FB70000E9467FC0895CF93DF9380914202909199
:10FB8000430297FF03C081E08BBF01C01BBEC0E0F2
:10FB9000D0E011C0AE014E5B5E4F80914202909169
:10FBA0004302880F991F60E071E08C0F9D1F0E9437
:10FBB0007EFCC050DF4F8091400190914101C817F9
:10FBC000D90740F30E94D6FCDF91CF9108950E949F
:10FBD00006FD8823E1F30E9403FD803211F481E0E9
:10FBE000089585E10E94F7FC80E00895DF92EF928E
:10FBF000FF920F931F93CF93DF9369E081E090E032
:10FC00000E94C7FC84FF03C08F7E0E94BEFCDD24DF
:10FC10000E9406FD8823E1F30E9403FD8235C0F4B3
:10FC2000803508F078C0813409F443C0823448F448
:10FC3000813321F1803409F452C1803309F04BC182
:10FC40006AC0823409F458C0853409F044C157C0F1
:10FC5000863509F40DC1873538F4823509F461C061
:10FC6000853509F038C16CC0843709F4A6C08537E2
:10FC700009F4EEC0843609F02EC17AC00E94E7FD77
:10FC8000882331F284E10E94F7FC81E40E94F7FCB2
:10FC900086E50E94F7FC82E50E94F7FC80E20E9464
:10FCA000F7FC83E50E94F7FC84E50E94F7FC8BE4F7
:10FCB0000EC161E070E080E091E00E940AFD0E94C8
:10FCC000E7FD882309F4A4CF84E10E94F7FC80912A
:10FCD0000001813869F0823818F4803839F4C6C0E0
:10FCE000823841F0883911F483E0F1C080E0EFC040
:10FCF00081E0EDC082E1EBC064E170E008C061E04A
:10FD000070E080E091E00E940AFD64E070E080E035
:10FD100091E00E940AFD0E94E7FD882309F478CF54
:10FD20000DC00E94E7FD882309F472CF60E070E007
:10FD300080E090E00E94ABFC0E94D6FC84E1C7C04A
:10FD400062E070E080E091E00E940AFD0E94E7FD21
:10FD5000882309F45DCFF0900101EE248091000129
:10FD60009701280F311D3093430220934202E6CFC2
:10FD700063E070E080E091E00E940AFDD091000114
:10FD8000C0E080910101BE01680F711D70934101B7
:10FD90006093400182E491E00E940AFD0E94E7FD29
:10FDA000882309F435CF80910201863419F40E942A
:10FDB000BBFDC4CF0E944CFDC1CF63E070E080E08A
:10FDC00091E00E940AFD1091000100E08091010184
:10FDD0009801280F311D30934101209340010E946A
:10FDE000E7FD882309F414CF80910201863459F08D
:10FDF0004091400150914101609142027091430253
:10FE000020E030E010C00E94A5FD16C0C901860F99
:10FE1000971F9FBB8EBBE09A8DB3F901EE5BFE4F3F
:10FE200080832F5F3F4F2417350780F3460F571FFE
:10FE3000509343024093420284E10E94F7FC609198
:10FE400040017091410182E491E00E941FFD41C098
:10FE50000E94E7FD882309F4DBCE84E10E94F7FCD1
:10FE60008EE10E94F7FC87E90E94F7FC82E02FC038
:10FE700064E070E080E091E00E940AFD0E94E7FDEE
:10FE8000882309F4C5CE84E10E94F7FC809100012B
:10FE9000803531F480910101882359F4DD2412C0AA
:10FEA000883581F480910101883041F453E0D52EEA
:10FEB00009C0883039F442E0D42E04C0882311F4FC
:10FEC000DD24D39469E08D2D90E00E94C7FC0E9450
:10FED000F7FC80E101C085E10E94F7FC99CEDF913B
:10FEE000CF911F910F91FF90EF90DF9008950E94A6
:10FEF000F1FCE0E0F0E0099508951F93F894E19992
:10FF0000FECF8EEF9FE09FBB8EBBE09A8DB3843B0C
:10FF1000A1F4E199FECF8FEF9FE09FBB8EBBE09AEB
:10FF20008DB3833C51F4E199FECF8DEF9FE09FBBF1
:10FF30008EBBE09A8DB380936F000E94E8FC0E9414
:10FF400003FD1EE119C00000019648E08A3C9407B9
:10FF5000D1F72F5F3F4F2436310519F080E090E054
:10FF6000F2CF0E9406FD882319F00E94F6FD07C01B
:10FF7000115018BB112319F020E030E0EFCF0E94A0
:0EFF800077FF80E090E01F910895F894FFCF86
:040000031000F800F1
:00000001FF
